:100000008A1183125D2A0000772800308A002608B2
:100010008207FF34FE34FE34FE34FE34FE34FE34F8
:10002000EF34FE34FE34FE34FE34FE347F34FE34CE
:1000300067348134ED34433449342D341934113468
:10004000CD3401340934FF347F34FB34FE340034C2
:10005000FE34FE34053431347334613413341734D0
:1000600091343534B734E1343334B33485347534B2
:10007000713407340D34773419349734F134A134A2
:100080005B34253429347B34FE34FE34FE34FE34B4
:10009000FE34FB3405343134733461341334173493
:1000A00091343534B734E1343334B3348534753472
:1000B000713407340D34773419349734F134A13462
:1000C0005B34253429347B34FE34FE34FE34FE3474
:1000D000FE3400308A002608820780344034203401
:1000E0001034083404340234003400340034000086
:1000F000A000030E8312A1000408A2000A08A300B6
:1001000000308A008C1F86280D218A288B1C8F289E
:100110005D218A288316891283128C138B10831217
:100120002208840023088A00210E8300A00E200EDE
:100130000900FB0D7B10051A7B14C0307B06031DE4
:10014000C428FD0A05307D06031DA8280130FD00E6
:1001500000308A0003107D0DA700270D82070030B4
:10016000F4004930C3280030F4004930C328083077
:10017000F4005130C3281030F4005930C32818302F
:10018000F4006130C328FC000800860187010510D7
:100190008510051108307306031DD4284808851EF4
:1001A000FF30870085140729FE0FD728FF0A093082
:1001B0007306031DEC287D08103EA6000520A6004E
:1001C0002609851AE728FF308700051507297F1AB9
:1001D00000308700051507297C0873078400FF306D
:1001E000801BFE30E90020300002031C1A30851EFF
:1001F0001E30A600A6130520E905690987007308CB
:10020000A600692086000730730603190514F30A57
:100210000A3073060319F30108000808F700F718FD
:100220005B2972107718721472087106031DF501AC
:100230007208F1007708F03975182129F600F60EDA
:100240005B29F604F60E771C332926292830840012
:100250007408840776088000F40A20307406031DB1
:100260003229F4015B29F608031947297608303949
:10027000203A031946297608C039803A03195229D1
:100280007608C039C03A031956295B295B29283002
:1002900084002030A40020308000840AA40B4C2964
:1002A000F4015B2976080F39F4005B2976080F39D1
:1002B000103EF4005B29F50A08003930F500F50B13
:1002C0005F290830F6000000F80C06186929F813B9
:1002D0006A29F8176B29000000002630F500F50B9D
:1002E0006F29F60B63292830F500F50B752977186F
:1002F000582A003078060319072A013078060319B6
:10030000172A0230780603191D2A033078060319CC
:10031000232A043078060319292A053078060319A0
:10032000562A0930780603193A2A0A307806031942
:10033000412A0B3078060319482A0C307806031935
:100340004F2A203078060319D0292D30780603195A
:10035000D0292E307806031DCB29F403073074060C
:10036000031DB4290F30F4000F307406031DBA29A1
:100370001730F40017307406031DC0291F30F40035
:10038000FF307406031DC6290730F4007408283EA8
:1003900084008017D52978082F3C031CD0295C2ABB
:1003A00028307407840078088000F40A01307D0644
:1003B000031DE1297408073C0318E0290030F4000C
:1003C0005C2A02307D06031DEC2974080F3C0318DB
:1003D000EB290830F4005C2A03307D06031DF72961
:1003E0007408173C0318F6291030F4005C2A043016
:1003F0007D06031D022A74081F3C0318012A1830C9
:10040000F4005C2A0130FD000030F4005C2A283042
:1004100084002030A40020308000840AA40B0C2A21
:100420000130FD004930FC000030F4005C2A01304E
:10043000FD004930FC0000302F2A0230FD00513011
:10044000FC0008302F2A0330FD005930FC0010302A
:100450002F2A0430FD006130FC0018302F2AF400F0
:10046000283E84000830A40020308000840AA40BB9
:10047000352A5C2A0130FD004930FC000030F400D0
:100480005C2A0230FD005130FC000830F4005C2A88
:100490000330FD005930FC001030F4005C2A0430B9
:1004A000FD006130FC001830F4005C2A77145C2AEF
:1004B0007808C80077105C2A08002030840080018A
:1004C000840A0408803A031D5F2AFF3085008600F5
:1004D0008700880089008316F83085000130860087
:1004E00000308700FF30880017308900803081009D
:1004F0008312F3012030A5002830840020308000D2
:10050000840AA50B7F2A0030C8000130FD00493065
:10051000FC0083168C170B170B168B178312010820
:10052000F9007A0879020319992A0318992AC52033
:1005300099207908FA00851D9E2A532B2D30D90069
:10054000DA00DB00DC00DD00DE00DF00E000E100BF
:10055000E200E300E400E500E600E700E8004130E7
:100560002806031DD12A42303806031DD12A6D30DA
:1005700029060319D12ABC2A5130FC000230FD00A3
:100580002030D1003108D2003208D3003308D40023
:100590002030D5004108D6004208D7004308D800D3
:1005A0008F2A4930FC000130FD00343084002E30A9
:1005B00000060030031DDE2A840380300004D000D2
:1005C00084032E3000060030031DE82A84038030A7
:1005D0000004CF0084032E3000060030031DF22AF1
:1005E000840380300004CE0084032E3000060030E7
:1005F000031DFC2A840380300004CD0084032E30C8
:1006000000060030031D062B840380300004CC005C
:1006100084032E3000060030031D102B840380302D
:100620000004CB0084032E3000060030031D1A2B7B
:10063000840380300004CA0084032E30000600309A
:10064000031D242B840380300004C900F030C8054A
:100650003508203A0319481435084B3A0319C814D1
:1006600035084D3A031948153508473A0319C81596
:100670000F30C8052808413A031948162808503A8F
:100680000319C8162808453A031D4A2B2B08413A7E
:10069000031948172808453A031D522B2B08423AE4
:1006A0000319C8178F2A2808C9002908CA002A0870
:1006B000CB002B08CC002C08CD002D08CE002E0836
:1006C000CF002F08D0003008D1003108D200320806
:1006D000D3003308D4003408D5003508D6003608D6
:1006E000D7003708D8003808D9003908DA003A08A6
:1006F000DB003B08DC003C08DD003D08DE003E0876
:10070000DF003F08E0004008E1004108E200420845
:10071000E3004308E4004408E5004508E600460815
:10072000E7004708E8008F2AFA30B22B0130A82BE7
:100730000230A82B0530A82B0A30A82B0F30A82B8D
:100740001430A82B2830A82B3230A82B6430A82BCB
:10075000EE00D030B223D030B223D030B223EE0B33
:0E076000A92B0800EF006400EF0BB32B08007C
:02400E00B23FBF
:00000001FF
